:1000000012C01EC118951895189518951895189531
:100010001895189518951895189518951895189578
:100020001895189518958FE58DBFC0E4E0E44E2E25
:1000300084E08EBFD4E0F4E05F2EEEEFF3E0A0E6C4
:10004000B0E088278D933197E9F784B7082E877F32
:1000500084BF8FE181BD87E081BD41DB662488E7F5
:1000600081BB86EC84BB8FE387BB80E082BB80E0F2
:1000700085BB80EC88BB929A969A789416DB8CE0CC
:1000800076DBE0E1F9E109DBE1E0F0E01FDB0BDB2F
:10009000E0E2F9E102DB84EF91E095DBE6E2F9E1F1
:1000A000FCDA84EF91E08FDBECE2F9E1F6DA8AEF3B
:1000B00090E089DBEEE2F9E1F0DA8AEF90E083DBB1
:1000C000E0E3F9E1EADA8AEF90E07DDBE2E3F9E1EF
:1000D000E4DA8AEF90E077DBE4E3F9E1DEDA8AEF55
:1000E00090E071DBE6E3F9E1D8DA8AEF90E06BDBD0
:1000F000E8E3F9E1D2DA8AEF90E065DBEAE3F9E1DF
:10010000CCDAE3E0F0E0E2DAD0DAECE3F9E1C5DA08
:10011000CADAECE3F9E1C1DAE2E0F0E0D7DAC5DA15
:10012000ECE4F9E1BADABFDAECE5F9E1B6DAE2E0FB
:10013000F0E0CCDABADAA6E3B0E00C9106FB81E09D
:100140000EF080E08F93A6E3B0E00C9107FB81E016
:100150000EF080E09F918923882309F403C081E099
:1001600080937100A6E3B0E00C9106FB81E00EF4F1
:1001700080E08F93A6E3B0E00C9107FB81E00EF0E6
:1001800080E09F918923882309F403C082E0809353
:100190007100A6E3B0E00C9106FB81E00EF080E078
:1001A0008F93A6E3B0E00C9107FB81E00EF480E0B2
:1001B0009F918923882309F403C083E08093710011
:1001C000A6E3B0E00C9106FB81E00EF480E08F9393
:1001D000A6E3B0E00C9107FB81E00EF480E09F9174
:1001E0008923882309F403C084E08093710000917F
:1001F0007100013009F003C0ECE6F9E14EDA00913C
:100200007100023009F003C0EAE7F9E146DA009133
:100210007100033009F003C0ECE8F9E13EDA009127
:100220007100043009F003C0EEE9F9E136DA8BB76A
:1002300080648BBF85B78F7D806A85BF88957BCFB3
:100240008BB78F7B8BBFEDEFF1E0ABE6B0E091E0D9
:1002500058DB00916B000E3C08F02AC026DA0091B2
:100260007100013009F003C0E0EBF9E116DA00910A
:100270007100023009F003C0E2ECF9E10EDA0091FE
:100280007100033009F003C0E4EDF9E106DA0091F2
:100290007100043009F003C0E6EEF9E1FED903DA9B
:1002A000E0E1F9E1FAD985B78F7D806A85BF88954D
:1002B00084E690E088DAA6E3B0E00C9106FB81E0EA
:1002C0000EF080E08F93A6E3B0E00C9107FB81E095
:1002D0000EF080E09F918923882309F403C081E018
:1002E00080937100A6E3B0E00C9106FB81E00EF470
:1002F00080E08F93A6E3B0E00C9107FB81E00EF065
:1003000080E09F918923882309F403C082E08093D1
:100310007100A6E3B0E00C9106FB81E00EF080E0F6
:100320008F93A6E3B0E00C9107FB81E00EF480E030
:100330009F918923882309F403C083E0809371008F
:10034000A6E3B0E00C9106FB81E00EF480E08F9311
:10035000A6E3B0E00C9107FB81E00EF480E09F91F2
:100360008923882309F403C084E080937100819974
:1003700001C0A3D3829919C0969888E290E023DA4D
:10038000A99AAA9A8AE090E01EDAAA988AE090E0F8
:100390001ADAA998AA9A8AE090E015DAAA989899A8
:1003A00001C07ED2989B01C065D4189508957DD96F
:1003B00000917100013009F003C0E8EFF9E16DD957
:1003C00000917100023009F003C0E6E0FAE165D95E
:1003D00000917100033009F003C0E4E1FAE15DD956
:1003E00000917100043009F003C0E4E2FAE155D94C
:1003F000EEEFF1E0ADE6B0E081DA00916D0041E0B2
:10040000040FAAE6B0E00C93A0E3B0E00C9100FB6F
:1004100081E00EF080E08F93A3E3B0E00C9105FB48
:1004200081E00EF080E09F918923882309F403C0C6
:1004300088E080937000A0E3B0E00C9100FB81E0C5
:100440000EF480E08F93A3E3B0E00C9105FB81E014
:100450000EF080E09F918923882309F403C080E196
:1004600080937000A0E3B0E00C9100FB81E00EF0FF
:1004700080E08F93A3E3B0E00C9105FB81E00EF4E4
:1004800080E09F918923882309F403C088E1809349
:100490007000A0E3B0E00C9100FB81E00EF480E07E
:1004A0008F93A3E3B0E00C9105FB81E00EF480E0B4
:1004B0009F918923882309F403C080E28093700010
:1004C0004091700000916A00041710F009F001C01B
:1004D00070C080E080936D00EEEFF1E0ADE6B0E03B
:1004E0007BE7FBD9969A8AEF8093650084E080933E
:1004F000670084D8DAD800917100013009F003C098
:10050000E6E3FAE1CAD800917100023009F003C0B5
:10051000E4E4FAE1C2D800917100033009F003C0AD
:10052000E2E5FAE1BAD800917100043009F003C0A5
:10053000E2E6FAE1B2D8009170000A3008F003C098
:10054000EEE2F9E1AAD8A8E2B4E0E0E7F0E075D97C
:100550009CD8A9D800917100013009F003C0E0E7F0
:10056000FAE19BD800917100023009F003C0E2E883
:10057000FAE193D800917100033009F003C0E4E977
:10058000FAE18BD800917100043009F003C0E4EA6D
:10059000FAE183D88AEF8093650084E08093670056
:1005A0002DD8829901C0FDCF80D884E690E00BD988
:1005B000089579D8969A00917100013009F003C02E
:1005C000ECE6F9E16AD800917100023009F003C04D
:1005D000EAE7F9E162D800917100033009F003C045
:1005E000E4EBFAE15AD800917100043009F003C03D
:1005F000E4ECFAE152D88AEF8093650080E08093C2
:100600006700FCD7829901C0FDCFA0E3B0E08C91D8
:1006100082FBDEF7A0E3B0E08C9182FBDEF39698DC
:1006200088E290E0D0D8A99AAA9A8AE090E0CBD844
:10063000AA988AE090E0C7D8A998AA9A8AE090E0A0
:10064000C2D8AA9881E080936100009161000F30C8
:1006500010F009F083C000916100023009F02AC057
:10066000009160000F3F09F025C01FD80091710074
:10067000013009F003C0E4EDFAE10FD800917100F8
:10068000023009F003C0E2EEFAE107D800917100F0
:10069000033009F003C0E2EFFAE1FFD700917100E7
:1006A000043009F003C0E2E0FBE1F7D7E2E0F0E05C
:1006B0000DD86FC780E08093600080E08093620077
:1006C00000916200073010F009F01FC0A0E6B0E012
:1006D0000C9142E0049F0C9200916000A3E3B0E013
:1006E0008C9183FB882780F9482F040FA0E6B0E0A7
:1006F0000C93AA9A8AE090E066D8AA98A2E6B0E0A5
:100700008C918F5F8C9308F4DBCFAAE6B0E00D915B
:1007100011274FE050E066D8A3E6B0E00D931C939C
:10072000A3E6B0E00D911C91A1E6B0E04D915527F4
:10073000040F151FA3E6B0E00D931C93A3E6B0E0F1
:10074000ED91FC91A0E6B0E091E07BE7C9D8A1E68D
:10075000B0E08C918F5F8C9308F477CFEEEFF1E0EF
:10076000AAE6B0E07BE7B9D884E690E02CD8969A68
:100770008AEF8093650081E08093670096D70091AF
:100780007100013009F003C0E2E1FBE186D700917E
:100790007100023009F003C0ECE1FBE17ED700916B
:1007A0007100033009F003C0E6E2FBE176D7009167
:1007B0007100043009F003C0E0E3FBE16ED7009163
:1007C0006A000A3008F003C0EEE2F9E166D7A8E259
:1007D000B4E0EAE6F0E031D858D70091710001307A
:1007E00009F003C0EAE3FBE158D700917100023041
:1007F00009F003C0E0E4FBE150D700917100033041
:1008000009F003C0E6E4FBE148D700917100043031
:1008100009F003C0ECE4FBE140D7009170000A301E
:1008200008F003C0EEE2F9E138D7A8E2B4E0E0E76F
:10083000F0E003D82AD737D700917100013009F0D2
:1008400003C0E2E5FBE129D700917100023009F015
:1008500003C0EEE5FBE121D700917100033009F000
:1008600003C0EAE6FBE119D700917100043009F0FA
:1008700003C0E8E7FBE111D7C1D6829901C0FDCFE3
:1008800014D7E1E0F0E022D786E98093650000917B
:100890006A0041E0041BA7E6B0E00C93AFD60895D0
:1008A00004D700917100013009F003C0E4E8FBE1D6
:1008B000F4D600917100023009F003C0E0E9FBE1D9
:1008C000ECD600917100033009F003C0ECE9FBE1C4
:1008D000E4D600917100043009F003C0E8EAFBE1BE
:1008E000DCD6E1D600917100013009F003C0E4EBE1
:1008F000FBE1D3D600917100023009F003C0E2ECB5
:10090000FBE1CBD600917100033009F003C0E2EDAA
:10091000FBE1C3D600917100043009F003C0E0EEA2
:10092000FBE1BBD684EF91E04ED781E0809361007C
:10093000009161000F3010F009F06AC00091610071
:10094000023009F02AC0009160000F3F09F025C075
:10095000ACD600917100013009F003C0E4EDFAE17A
:100960009CD600917100023009F003C0E0EFFBE17A
:1009700094D600917100033009F003C0E2EFFAE170
:100980008CD600917100043009F003C0E2E0FBE175
:1009900084D6E2E0F0E09AD6FCC580E08093600067
:1009A00080E08093620000916200073010F009F04F
:1009B0001FC0A0E6B0E00C9142E0049F0C920091B1
:1009C0006000A3E3B0E08C9183FB882780F9482F77
:1009D000040FA0E6B0E00C93AA9A8AE090E0F3D668
:1009E000AA98A2E6B0E08C918F5F8C9308F4DBCFDD
:1009F000A1E6B0E0EC91FF27A0E6B0E091E07BE754
:100A00006FD7A1E6B0E08C918F5F8C9308F490CF04
:100A100084E690E0D8D6969A8AEF8093650081E0CC
:100A20008093670042D600917100013009F003C045
:100A3000E4EBFBE132D600917100023009F003C013
:100A4000E0E0FCE12AD600917100033009F003C018
:100A5000E2EDFBE122D600917100043009F003C001
:100A6000E0EEFBE11AD61FD600917100013009F0CB
:100A700003C0E2E5FBE111D600917100023009F0FC
:100A800003C0EEE5FBE109D600917100033009F0E7
:100A900003C0EAE6FBE101D600917100043009F0E1
:100AA00003C0E0E1FCE1F9D5A9D5829901C0FDCFF1
:100AB000989901C0FACFF9D50895F7D50091710042
:100AC000013009F003C0EEE1FCE1E7D500917100CF
:100AD000023009F003C0EEE2FCE1DFD500917100C5
:100AE000033009F003C0EEE3FCE1D7D500917100BB
:100AF000043009F003C0EEE4FCE1CFD5D4D5009179
:100B00007100013009F003C0EEE5FCE1C6D50091AB
:100B10007100023009F003C0EEE6FCE1BED50091A1
:100B20007100033009F003C0ECE7FCE1B6D5009199
:100B30007100043009F003C0ECE8FCE1AED581E0BF
:100B400080936F0080E190E0A8E6B0E08D939C93E5
:100B5000A8E6B0E00D911C910C3F51E0150710F094
:100B600009F02AC000916F00083F09F003C080E33C
:100B70008093670000916700003309F005C0809101
:100B80006F00815080936F0000916700003309F47B
:100B900005C0AFE6B0E08C918F5F8C93A8E6B0E023
:100BA000ED91FC91AFE6B0E091E07BE799D6A8E645
:100BB000B0E043D508F4CCCF80E080936D00EEEF39
:100BC000F1E0ADE6B0E07BE788D684E690E0FBD5C7
:100BD000969A8AEF8093650082E08093670065D5DE
:100BE00000917100013009F003C0EAE9FCE155D53C
:100BF00000917100023009F003C0EAEAFCE14DD532
:100C000000917100033009F003C0ECEBFCE145D525
:100C100000917100043009F003C0ECECFCE13DD51B
:100C200042D500917100013009F003C0ECEDFCE108
:100C300034D500917100023009F003C0EEEEFCE102
:100C40002CD500917100033009F003C0E0E0FDE114
:100C500024D500917100043009F003C0E2E1FDE108
:100C60001CD5CCD4829901C0FDCF819901C0FACFA7
:100C70001CD5089580E080936F0017D58FE711E0B1
:100C800023D500917100013009F003C0E4E2FDE1D9
:100C900004D500917100023009F003C0E2E3FDE1E8
:100CA000FCD400917100033009F003C0E0E4FDE1E1
:100CB000F4D400917100043009F003C0ECE4FDE1CC
:100CC000ECD484EF91E07FD581E0809361000091C6
:100CD00061000F3010F009F0E5C380E08093600000
:100CE00080E08093620000916200073010F009F00C
:100CF0001CC0A0E6B0E00C9142E0049F0C92009171
:100D00006000A3E3B0E08C9183FB882780F9482F33
:100D1000040FA0E6B0E00C93AA9AAA98A2E6B0E06D
:100D20008C918F5F8C9308F4DECFA1E6B0E0EC915C
:100D3000FF27A6E6B0E091E0E4D54091660000917F
:100D40006000041709F401C006C0AFE6B0E08C9162
:100D50008F5F8C93A0C3A1E6B0E00D9111274FE007
:100D600050E0040F151FA3E6B0E00D931C93A3E61B
:100D7000B0E0ED91FC91A6E6B0E091E0C2D54091E3
:100D8000660000916000041709F401C001C083C32C
:100D9000A1E6B0E00D9111274EE150E0040F151FC0
:100DA000A3E6B0E00D931C93A3E6B0E0ED91FC91B7
:100DB000A6E6B0E091E0A5D5409166000091600004
:100DC000041709F401C001C066C3A1E6B0E00D91AB
:100DD00011274DE250E0040F151FA3E6B0E00D937C
:100DE0001C93A3E6B0E0ED91FC91A6E6B0E091E0A3
:100DF00088D54091660000916000041709F401C095
:100E000001C049C3A1E6B0E00D9111274CE350E0C9
:100E1000040F151FA3E6B0E00D931C93A3E6B0E00A
:100E2000ED91FC91A6E6B0E091E06BD540916600B3
:100E300000916000041709F401C001C02CC3A1E6B1
:100E4000B0E00D9111274BE450E0040F151FA3E60D
:100E5000B0E00D931C93A3E6B0E0ED91FC91A6E603
:100E6000B0E091E04ED5409166000091600004171B
:100E700009F401C001C00FC3A1E6B0E00D91112734
:100E80004AE550E0040F151FA3E6B0E00D931C9354
:100E9000A3E6B0E0ED91FC91A6E6B0E091E031D59B
:100EA0004091660000916000041709F401C001C080
:100EB000F2C2A1E6B0E00D91112749E650E0040F1F
:100EC000151FA3E6B0E00D931C93A3E6B0E0ED91EF
:100ED000FC91A6E6B0E091E014D540916600009147
:100EE0006000041709F401C001C0D5C2A1E6B0E05A
:100EF0000D91112748E750E0040F151FA3E6B0E05D
:100F00000D931C93A3E6B0E0ED91FC91A6E6B0E052
:100F100091E0F7D44091660000916000041709F455
:100F200001C001C0B8C2A1E6B0E00D91112747E8A9
:100F300050E0040F151FA3E6B0E00D931C93A3E649
:100F4000B0E0ED91FC91A6E6B0E091E0DAD44091FA
:100F5000660000916000041709F401C001C09BC243
:100F6000A1E6B0E00D91112746E950E0040F151FEE
:100F7000A3E6B0E00D931C93A3E6B0E0ED91FC91E5
:100F8000A6E6B0E091E0BDD440916600009160001B
:100F9000041709F401C001C07EC2A1E6B0E00D91C2
:100FA000112745EA50E0040F151FA3E6B0E00D93AA
:100FB0001C93A3E6B0E0ED91FC91A6E6B0E091E0D1
:100FC000A0D44091660000916000041709F401C0AC
:100FD00001C061C2A1E6B0E00D91112744EB50E0E1
:100FE000040F151FA3E6B0E00D931C93A3E6B0E039
:100FF000ED91FC91A6E6B0E091E083D440916600CB
:1010000000916000041709F401C001C044C2A1E6C8
:10101000B0E00D91112743EC50E0040F151FA3E63B
:10102000B0E00D931C93A3E6B0E0ED91FC91A6E631
:10103000B0E091E066D44091660000916000041732
:1010400009F401C001C027C2A1E6B0E00D9111274B
:1010500042ED50E0040F151FA3E6B0E00D931C9382
:10106000A3E6B0E0ED91FC91A6E6B0E091E049D4B2
:101070004091660000916000041709F401C001C0AE
:101080000AC2A1E6B0E00D91112741EE50E0040F35
:10109000151FA3E6B0E00D931C93A3E6B0E0ED911D
:1010A000FC91A6E6B0E091E02CD44091660000915E
:1010B0006000041709F401C001C0EDC1A1E6B0E071
:1010C0000D91112740EF50E0040F151FA3E6B0E08B
:1010D0000D931C93A3E6B0E0ED91FC91A6E6B0E081
:1010E00091E00FD44091660000916000041709F46C
:1010F00001C001C0D0C1A1E6B0E00D9111274FEFB2
:1011000050E0040F151FA3E6B0E00D931C93A3E677
:10111000B0E0ED91FC91A6E6B0E091E0F2D3409111
:10112000660000916000041709F401C001C0B3C15A
:10113000A1E6B0E00D9111274EE051E0040F151F1C
:10114000A3E6B0E00D931C93A3E6B0E0ED91FC9113
:10115000A6E6B0E091E0D5D3409166000091600032
:10116000041709F401C001C096C1A1E6B0E00D91D9
:1011700011274DE151E0040F151FA3E6B0E00D93D8
:101180001C93A3E6B0E0ED91FC91A6E6B0E091E0FF
:10119000B8D34091660000916000041709F401C0C3
:1011A00001C079C1A1E6B0E00D9111274CE251E0F8
:1011B000040F151FA3E6B0E00D931C93A3E6B0E067
:1011C000ED91FC91A6E6B0E091E09BD340916600E2
:1011D00000916000041709F401C001C05CC1A1E6E0
:1011E000B0E00D9111274BE351E0040F151FA3E66A
:1011F000B0E00D931C93A3E6B0E0ED91FC91A6E660
:10120000B0E091E07ED34091660000916000041749
:1012100009F401C001C03FC1A1E6B0E00D91112762
:101220004AE451E0040F151FA3E6B0E00D931C93B0
:10123000A3E6B0E0ED91FC91A6E6B0E091E061D3C9
:101240004091660000916000041709F401C001C0DC
:1012500022C1A1E6B0E00D91112749E551E0040F4C
:10126000151FA3E6B0E00D931C93A3E6B0E0ED914B
:10127000FC91A6E6B0E091E044D340916600009175
:101280006000041709F401C001C005C1A1E6B0E087
:101290000D91112748E651E0040F151FA3E6B0E0B9
:1012A0000D931C93A3E6B0E0ED91FC91A6E6B0E0AF
:1012B00091E027D34091660000916000041709F483
:1012C00001C001C0E8C0A1E6B0E00D91112747E7D9
:1012D00051E0040F151FA3E6B0E00D931C93A3E6A5
:1012E000B0E0ED91FC91A6E6B0E091E00AD3409128
:1012F000660000916000041709F401C001C0CBC072
:10130000A1E6B0E00D91112746E851E0040F151F4A
:10131000A3E6B0E00D931C93A3E6B0E0ED91FC9141
:10132000A6E6B0E091E0EDD2409166000091600049
:10133000041709F401C001C0AEC0A1E6B0E00D91F0
:10134000112745E951E0040F151FA3E6B0E00D9306
:101350001C93A3E6B0E0ED91FC91A6E6B0E091E02D
:10136000D0D24091660000916000041709F401C0DA
:1013700001C091C0A1E6B0E00D91112744EA51E00F
:10138000040F151FA3E6B0E00D931C93A3E6B0E095
:10139000ED91FC91A6E6B0E091E0B3D240916600F9
:1013A00000916000041709F401C001C074C0A1E6F7
:1013B000B0E00D91112743EB51E0040F151FA3E698
:1013C000B0E00D931C93A3E6B0E0ED91FC91A6E68E
:1013D000B0E091E096D24091660000916000041761
:1013E00009F401C001C057C0A1E6B0E00D9111277A
:1013F00042EC51E0040F151FA3E6B0E00D931C93DF
:10140000A3E6B0E0ED91FC91A6E6B0E091E079D2E0
:101410004091660000916000041709F401C001C00A
:101420003AC0A1E6B0E00D91112741ED51E0040F63
:10143000151FA3E6B0E00D931C93A3E6B0E0ED9179
:10144000FC91A6E6B0E091E05CD24091660000918C
:101450006000041709F401C001C01DC0A1E6B0E09E
:101460000D91112740EE51E0040F151FA3E6B0E0E7
:101470000D931C93A3E6B0E0ED91FC91A6E6B0E0DD
:1014800091E03FD24091660000916000041709F49A
:1014900001C07FC000C0A1E6B0E08C918F5F8C934B
:1014A00008F415CC00916F000E3010F009F001C067
:1014B00001C07DC7FAD0F7D000917100013009F06A
:1014C00003C0ECE5FDE1E9D000917100023009F0C4
:1014D00003C0ECE6FDE1E1D000917100033009F0BA
:1014E00003C0EEE7FDE1D9D000917100043009F0AE
:1014F00003C0EEE8FDE1D1D0969A8AEF80936500B3
:1015000081E0809367007AD0829901C0FDCFCDD071
:10151000CAD000917100013009F003C0E0EAFDE19A
:10152000BCD000917100023009F003C0EEEAFDE189
:10153000B4D000917100033009F003C0ECEBFDE181
:10154000ACD000917100043009F003C0EAECFDE179
:10155000A4D0E1E0F0E0BAD0949AE2E0F0E0B6D0B6
:101560009498A3D0E0E1F9E198D0E2E0F0E0AED0C9
:1015700080916B00815080936B00EDEFF1E0ABE662
:10158000B0E091E07BE7ACD190D0E1E0F0E09ED01C
:1015900008958BD000917100013009F003C0E8ED8F
:1015A000FDE17BD000917100023009F003C0E6EE4E
:1015B000FDE173D000917100033009F003C0E6EF44
:1015C000FDE16BD000917100043009F003C0E6E04A
:1015D000FEE163D068D0E0E1F9E15FD0969A8AE558
:1015E0008093650089E08093670008D0829901C0EC
:1015F000FDCFE1E0F0E06AD058D0089580E080931C
:1016000061004091670000916100041710F009F03B
:1016100013C0939AA5E6B0E08C919927D4D0939803
:10162000A5E6B0E08C919927CED0A1E6B0E08C91F0
:101630008F5F8C9308F4E5CF0895ED91FC91EF5FF7
:10164000FF4FFC93EE93089504D0CCD000FC0CD057
:1016500008950024E89457FF02C009D0689400F868
:101660000BD010F80124089502D009D008955095A8
:1016700040954F5F5F4F0895E89417FF08950095D8
:1016800010950F5F1F4F68940895A8E2B4E08D9104
:10169000882311F066D0FBCF0895AED0802D11F0D5
:1016A00060D0FBCF089580EC62C081E060D014D0A0
:1016B00080E85DC08FE7213039F08FEB223021F0D8
:1016C0008FE8233009F08FEC810F51C088EE93E052
:1016D0007AD03197D9F7089583E0992774C08AEFBB
:1016E00090E071D0BD9ABC9ABB9ABA9AB99AB89A4E
:1016F000C09885E090E067D0C198C598C498C39A17
:10170000C29AC19AEF93FF93E5E1F0E050D0FF91C8
:10171000EF91C19855D0C19AEF93FF93E5E1F0E0C6
:1017200046D0FF91EF91C1984BD0C19AEF93FF93B0
:10173000E5E1F0E03CD0FF91EF91C19841D0C29833
:10174000C19AEF93FF93E5E1F0E031D0FF91EF9183
:10175000C19836D088E20BD08EE009D086E007D061
:101760000895C09A829505D004D02AD00895C098D3
:10177000F9CF859510F4C29A01C0C298859510F4EE
:10178000C39A01C0C398859510F4C49A01C0C49847
:10179000859510F4C59A01C0C598C19AEF93FF933F
:1017A000E5E1F0E004D0FF91EF91C1980895319701
:1017B000F1F70895689462F80895E89462F808953E
:1017C00081E090E000C0EF93FF93EE27E82BE92B38
:1017D00031F0EAEFF0E03197F1F70197D1F7FF919F
:1017E000EF9108950F92B801469F8001479F100D19
:1017F000569F100D0F900895C895319600200895BA
:10180000000F111F221F331F08950095109520957A
:1018100030950F5F1F4F2F4F3F4F0895019110815B
:101820000EC001911191219130810BC00191108165
:1018300017FF05C03FEF2FEF04C0008111272227BB
:10184000332737FF03C0E1DF8DE28D93CF93DF9322
:10185000CF92DF92EF92AA24BB24CC24DD24EE2485
:1018600040E2CAE0DD2755E093E38881890F87FDD8
:101870009F7083FD907F891B89935A95A9F7C0DFDC
:10188000AA1CBB1CCC1CDD1CEE1C4A9551F7E8942D
:10189000EFE0FF2782910ED0EB30E0F71EF0689466
:1018A0008A2D0CD088278D93EF90DF90CF90DF9119
:1018B000CF910895982F829501D0892F8F70805DE8
:1018C00026F0803309F4089568948D930895E19982
:1018D000FECFEEBBFFBB3196089591E001C092E0D0
:1018E0007B3751F47FB7F894F2DF8D918DBBE29A8C
:1018F000E19A9A95C9F77FBF7727089591E001C0D3
:1019000092E0E5DFE09A8DB38D939A95D1F7089533
:101910005757572E4156522E344D472E434F4D00A8
:1019200047534D3A00002B33383600003400300066
:101930003800330032003100370039005345542F4E
:101940004E4153544156493D3E51310030303D45A2
:101950004E47202C2031303D534C4F0030313D4715
:101960004552202C2031313D455350002020496EF6
:101970007365727420436172640056737461766992
:101980007465206B61727469636F0000496E7365E2
:10199000727420436172642D474552200000496EE5
:1019A0007365727420436172642D455350200000AA
:1019B000212044454D4F204558504952454420214F
:1019C0000000212044454D4F20504F54454B454C7D
:1019D0002021000044454D4F204558504952454470
:1019E0002D474552000044454D4F2045585049521F
:1019F00045442D455350000057726974696E672045
:101A000043617264000056706973206B617274697F
:101A1000636500005363687265696265204B61729B
:101A20007465000047726162616E646F2074617258
:101A30006A65746100004D656D6F72792066756C22
:101A40006C3A000053706F6D696E20706F6C6E3A67
:101A50000000537065696368657220766F6C6C3A3C
:101A6000000053696E206D656D6F7269613A000008
:101A700057726974696E6720436172643D3E30310C
:101A8000000056706973206B6172746963653D3E36
:101A9000303100005363687265696265204B2E3DEA
:101AA0003E303100477261622E207461726A2E3DB1
:101AB0003E3031004B617274652065696E66FC686A
:101AC00072656E00496E7365727465207461726A26
:101AD000657461002020205475726E204361726429
:101AE00000004F62726E697465206B617274696385
:101AF0006F0020204B617274652077656E64656E9F
:101B0000000020566F6C746565207461726A65749C
:101B1000610043617264204E6F3A00004B61727441
:101B20006963613A00004B617274654E723A00005D
:101B30005461726A6574613A0000206F662000008B
:101B4000206F6420000020766F6E200020646520E6
:101B50000000202020207772697474656E002020B8
:101B6000202076706973616E610020206765736361
:101B70006872696562656E0020202020677261626C
:101B80006164610020205772697474696E67000097
:101B9000202056706973756A656D00002053636874
:101BA00072656962656E0000202047726162616E35
:101BB000646F000020204D61737465722043617270
:101BC0006400204D6173746572206B617274696387
:101BD0006F00202048617570742D4B617274650030
:101BE0005461726A657461204D616573747261003D
:101BF000204F62726E69206B61727469636F0000BE
:101C0000204D6173746572206B6172746963610049
:101C100020202020206772616261646F00002045EF
:101C2000726173696E6720436172647300002042C1
:101C3000726973656D206B61727469636500204B16
:101C400061727465206CF6736368656E00002042F3
:101C50006F7272616E646F207461726A2E0020660A
:101C6000726F6D20303120746F20333200002020DD
:101C70006F642030312064302033320020766F6E64
:101C8000203031206269732033320000202020642C
:101C9000652030312061203332002043617264734B
:101CA0003A203031202D203332004B617274696349
:101CB000653A203031202D203332000020204B6146
:101CC0007274653A2030312D333200005461726AEB
:101CD000657461733A2030312D333200202020208A
:101CE0002020202065726173656420200000202080
:101CF0002020202020697A62726973616E6500007D
:101D0000202020202020202067656CF673636874F3
:101D10000000202020202020202020626F7272618D
:101D2000646F000020202020436865636B696E6744
:101D30000000202020205072657665726A616D0077
:101D400020202020205072FC66656E002020205646
:101D5000657269666963616E646F00002043617239
:101D60006420657863657074656400004B6172740B
:101D700069636120737072656A6574610000204B4D
:101D80006172746520657277617274657400546164
:101D9000726A2E20657863657074756164610000F5
:101DA00020202020556E6C6F636B6564000020203E
:101DB000204F646B6C656E6A656E6F002020204555
:101DC0006E7472696567656C7400202020446573C9
:101DD000747261626164610020202043617264203A
:101DE00077726F6E67004B617274696361206E6118
:101DF0007061636E61002046616C73636865204B9F
:101E0000617274650000205461726A6574612065B6
:061E1000727261646100C2
:00000001FF
